:0200000480007A
:100000006F000005732F2034930F80006308FF03F7
:10001000930F90006304FF03930FB0006300FF038E
:10002000130F000063040F0067000F00732F2034CC
:1000300063540F006F00400093E19153171F0000BD
:1000400023223FFC171F000023200FFC6FF01FFF2F
:100050009300000013010000930100001302000050
:100060009302000013030000930300001304000038
:100070009304000013050000930500001306000020
:100080009306000013070000930700001308000008
:10009000930800001309000093090000130A0000F0
:1000A000930A0000130B0000930B0000130C0000D8
:1000B000930C0000130D0000930D0000130E0000C0
:1000C000930E0000130F0000930F0000732540F102
:1000D0006310050097020000938202017390523072
:1000E000735044749702000093820201739052305F
:1000F00073500018970200009382020273905230EE
:10010000B70200809382F2FF7390023B9302F001EA
:100110007390023A7350403097020000938242017C
:100120007390523073502030735030309301000080
:1001300097020000938242ED739052301305100035
:100140001315F501634C05000F00F00F930110002B
:100150009308D0051305000073000000930200000F
:10016000638A020073905210B7B20000938292101B
:100170007390223073500030970200009382420146
:1001800073901234732540F17300203093012000E6
:100190009300000013D70040930300006314772AF4
:1001A00093013000B700008013D71040B70300C0A0
:1001B000631A772893014000B700008013D770407E
:1001C000B70300FF6310772893015000B700008049
:1001D00013D7E040B703FEFF631677269301600054
:1001E000B70000809380100013D7F0419303F0FF15
:1001F000631A772493017000B70000809380F0FFAA
:1002000013D70040B70300809383F3FF631C77226A
:1002100093018000B70000809380F0FF13D7104057
:10022000B70300409383F3FF631E77209301900090
:10023000B70000809380F0FF13D77040B703000130
:100240009383F3FF631077209301A000B700008031
:100250009380F0FF13D7E040B70302009383F3FFCE
:100260006312771E9301B000B70000809380F0FF07
:1002700013D7F041930300006316771C9301C0006D
:10028000B78081819380101813D70040B783818194
:10029000938313186318771A9301D000B780818174
:1002A0009380101813D71040B7C3C0C09383030CBA
:1002B000631A77189301E000B7808181938010184A
:1002C00013D77040B70303FF93833330631C771653
:1002D0009301F000B78081819380101813D7E0401C
:1002E000B703FEFF93836360631E771493010001DD
:1002F000B78081819380101813D7F0419303F0FFEA
:100300006312771493011001B700008093D07040FE
:10031000B70300FF639870129301200113020000DD
:10032000B700008013D770401303070013021200B8
:1003300093022000E31652FEB70300FF631473100C
:100340009301300113020000B700008013D7E04092
:100350001300000013030700130212009302200091
:10036000E31452FEB703FEFF631E730C93014001BA
:1003700013020000B70000809380100013D7F041F3
:100380001300000013000000130307001302120003
:1003900093022000E31052FE9303F0FF6314730AEC
:1003A0009301500113020000B700008013D7704082
:1003B0001302120093022000E31852FEB70300FF5D
:1003C000631277089301600113020000B7000080F8
:1003D0001300000013D7E040130212009302200024
:1003E000E31652FEB703FEFF631E7704930170010C
:1003F00013020000B700008093801000130000007B
:100400001300000013D7F0411302120093022000E2
:10041000E31252FE9303F0FF63167702930180010B
:100420009350404093030000639E7000930190013D
:100430009300100213D0A0409303000063147000D7
:10044000631030020F00F00F6380010093911100E0
:1004500093E111009308D00513850100730000009B
:100460000F00F00F930110009308D0051305000052
:0C04700073000000731000C000000000CA
:1010000000000000000000000000000000000000E0
:1010100000000000000000000000000000000000D0
:1010200000000000000000000000000000000000C0
:1010300000000000000000000000000000000000B0
:081040000000000000000000A8
:040000058000000077
:00000001FF
